:100000000C9437000C94AC000C94AC000C94AC0035
:100010000C94AC000C94AC000C94AC000C94AC00B0
:100020000C94AC000C947E000C94AC000C94AC00CE
:100030000C94AC000C94AC000C94AC000C94AC0090
:100040000C94AC000C94AC000C94AC000C94AC0080
:100050000C94AC000C94AC000C94AC000C94AC0070
:100060000C94AC000C94AC0001000103800011243E
:100070001FBECFEFD8E0DEBFCDBFE8E6F0E040E046
:1000800017C0B591A59135912591059107FD0CC03B
:1000900095918591EF01F92FE82F05900D92A21708
:1000A000B307D9F7FE0104C01D92A217B307E1F709
:1000B000ED36F40731F70E9461000C949B00F89430
:0200C000FFCF70
:1000C2000E9490008AB180668AB98AB180618AB939
:1000D2008BB180618BB987B1886087B984E00E9457
:1000E200A60080E28093B6001092B00081E0809377
:0A00F200B100809370007894FFCFF6
:1000FC001F920F920FB60F9211248F939F9398B16A
:10010C0088E0892788B99F918F910F900FBE0F902F
:04011C001F90189583
:1001200080E006C0E82FF0E0E050FF4F10828F5FC4
:060130008330C0F30895C6
:10013600EC010E94B1000E94B000CE010E94B20004
:06014600CE010E94AE0094
:0C014C009BB190649BB980930001089562
:040158000C94000003
:04015C000E945F009E
:02016000089500
:020162000895FE
:020164000895FC
:00000001FF
